:030000000219FDE5
:03000B000200AA46
:03002B0002015679
:03005B000202E2BC
:030073000202CFB7
:1000800002030406080C10182030406080040608A3
:100090000C10182030406080A0C00003070F1F0D17
:1000A0000D0403060D0502030202C2AFC0D0C0E07A
:1000B000206214E5256009E473E525F4F58AD2622F
:1000C000D0E0D0D0D2AF3285268AC262E526F46075
:1000D00029D0E0D0D0C294C292C290D2AF32C294A2
:1000E000C292C290206F0C2065097405D5E0FDE531
:1000F0007B4290D0E0D0D0D2AF32758A00C28DD290
:100100006201F301B9306805206502D29401B9306B
:100110006805206502D29201B9306805206502D2D7
:100120009001B9C29530680A2065077428D5E0FDB2
:10013000D29401B9C29330680A2065077428D5E0CB
:10014000FDD29201B9C29130680A2065077428D5A2
:10015000E0FDD29001B9C2AFC2AD53E6EFC0D0C04E
:10016000E0D2D3D2AFC2CEE52A6007207449152A67
:1001700021B77800790020742EE580307E01F430BC
:10018000E40278FF53DACF207E0343DA20307E0387
:1001900043DA10C2D8C271E580307E01F430E40247
:1001A00079FFC3E89970CB306103752A402074034E
:1001B000752A40885CD27020740DE52B6004152BE5
:1001C00021C743DA01C2D820700221DAA85C20617D
:1001D00002C27020740221D888227882B604038576
:1001E000222420CF0AD0E0D0D043E610D2AD32C2D4
:1001F000CF053A7802E52A6005307402152AC3E576
:100200005C94014005755F00411B756000756900D5
:10021000E55F2401F55F5003755FFF7982B7020D3A
:10022000306E1DC3E52294324016854C227982B788
:10023000030E306E0BC3E52294324004798E872280
:10024000C3E5239522600840041523414F0523D8B8
:10025000CA0569E56970021569D56A69756A017828
:1002600008E56B60497805C3E569956B4057C3E5C0
:1002700069956C50087801756A03020289C3E569C3
:10028000956D50057801756A01C3E5629524401E9D
:100290007982B7040241BA206E14852462E56904AC
:1002A0006003856B69756A0175233C0202C5E562CE
:1002B0002850057562FF41BAF562E5620470067563
:1002C00060FF7569FFD0E0D0D043E610D2AD32C2F6
:1002D000AF53E67F7592FA7593FFC260759104D2B1
:1002E000AF32C2AF53E6EFC2ADC0D0C0E0C0F0D273
:1002F000D3D2AFA8FBA9FCC2D8307102614953DA4E
:10030000CF207E0343DA10307E0343DA20D271E53A
:1003100080307E01F420E402612088278928A12E04
:1003200053DACF207E0343DA20307E0343DA10C253
:10033000D8C271307402A11A7800E580307E01F4D1
:1003400030E402A11A885CA10253DACF207E034375
:10035000DA20307E0343DA10C27120610281225319
:10036000DACF207E0343DA10307E0343DA20C2D88E
:10037000D27188578958C3E89555F8E99556F97BA5
:10038000007E087A00C3E8948CE994005005755B00
:10039000008114882178A2E6A8216055C3E894C89A
:1003A000E994005008E4D2E4FB7A0A61EFC3E894D0
:1003B00068E994015008E4D2E3FB7A0F61EFC3E8E7
:1003C00094D0E994025008E4D2E2FB7A1E61EFC3B4
:1003D000E894A0E994055008E4D2E1FB7A3C61EF8F
:1003E000C3E89498E994085008E4D2E0FB7A787E58
:1003F00000C3E89559FCE9955AFD30E70AECF4246E
:1004000001FCEDF43400FD755B00C3EC9AED9E50E9
:1004100003755B018859895A855755855856780266
:10042000A102C3E89527F8E99528F9307C0281E616
:10043000307B0281E6307A0281DF2075028145E956
:10044000FDE8FC8164E9C313F9E813F8307902810F
:10045000DFE9C313F9E813F830780281DFE9C31349
:10046000FDE813FC20612CC3EC941CED94024002C7
:0F047000817BED701EC3EC94C850180529E52957
:10047F0070021529C3E529940A5002A11A755C0070
:10048F00D270A11AE529600215297400207F037824
:10049F0096E624FAFEE43400FFC3EC9EFCED9FFDCC
:1004AF0050067800790081E6C3EC94FFED9400408C
:1004BF000678FF790081E6EC8572F0A4C5F0A2F70B
:1004CF0033F87900400302050278FF790002050234
:1004DF00E9C313F9E813F8307C0EE9600278FFC323
:1004EF00E81338F8E43400F9C3E894FFE9940040C6
:1004FF000278FF885CD270206102A11A741FF45534
:10050F002F4BF52FC274EB7002D274752A403074E2
:10051F0003752A0A306102A12E20740353DAFE20DC
:10052F007403752B20D0F0D0E0D0D0D2AD43E610BD
:10053F0032790102055E790302055E790A02055ED2
:10054F00791E02055E796402055E79C802055E7840
:10055F0017E4D5E0FDD8FAD9F6227A147B78020594
:10056F00857A107B8C0205857A0D7BB40205857A1E
:10057F000B7BC8020585E573D5E001227902E4C241
:10058F0093D5E0FDD292D5E0FDC292D5E0FDD29396
:10059F00D5E0FDE920E002D29430E002D290E5737D
:1005AF00D5E0FDE920E002C29430E002C2907496DB
:1005BF00D5E0FDD9C9EAF8D5E0FDD8FBDBB8C29389
:1005CF0022C37C007D0075F00005F0EA33FAEB33AF
:1005DF00FB50F6EB13FBEA13FAC3E9FFE8FEE89AC8
:1005EF00F8E99BF95004EFF9EEF8B3EC33FCED3377
:1005FF00FDD5F0DFEDF9ECF822E889F08A20D2D4AE
:10060F00F8A9F07B0030F70B7BFFF42401F8E9F435
:10061F003400F9E88520F0A4ADF0F8E98520F0A4C6
:10062F00AFF0FEED2EF974003FFA7C04C3EA13FA23
:10063F00E913F9E813F8DCF48BF030F70AE8F42447
:10064F0001F8E9F43400F9E889F0C2D4F8A9F022EE
:10065F007882B604030206FEC3E55C9419401EE5DA
:10066F002D54067018206E3678057994E7146007BC
:10067F00780A1460027812C3E54198401F306E0962
:10068F008564627569FF756A01852224E4F544F576
:10069F0045F546F547F548C26E0206FED26E7994CF
:1006AF00E7147013E523F43333F913F8E954010415
:1006BF00F9E854FE0206F2E714147014E523F4333C
:1006CF003333F913F8E9540304F9E854FC0206FA3A
:1006DF00E523F433333333F913F8E954070404F9FA
:1006EF00E854F8C39440F8E99400F9884489452206
:1006FF00C3E54113F9E54013F8C3E54498F8E54520
:10070F0099F9500CC3E89480E994FF40160207361C
:10071F00C3E8947FE994005003020736787F79008D
:10072F00020736788079FF8849894A22E5492546AC
:10073F00F8E54A3547F9854A20E4300701F4354892
:10074F00FA30E709C3EA94F04015020774C3EA943C
:10075F000F500302077478FF79FF7A0F020774783E
:10076F000079007AF0C3E5249561500AC3740195AE
:10077F0024500B020792E54A20E70E020792E54A42
:10078F0030E706884689478A482278A5E6FAC3E506
:10079F004933F8E54A33F9D108E930E70BC3E89458
:1007AF0080E994FF4013E1CCC3E8947FE9940050B3
:1007BF0002E1CC787F7900E1CC788079FFE820E7FF
:1007CF0015C3E52398F84009C3E8940140030207D5
:1007DF00F378010207F3E8F424012523F84003021C
:1007EF0007F378FF884B2278A6E6FAA847A94812A4
:1007FF000608E930E70CC3E89401E994FF401602BC
:10080F000828C3E894FFE99400500302082878FFF2
:10081F007900020828780179FFE920E715C3E54B35
:10082F0098F84009C3E89401400302084F78010289
:10083F00084FE8F42401254BF8400302084F78FFD6
:10084F0088242278FF20692879A1E76023E5416099
:10085F001F74FF8541F0848539F0306A0375F00508
:0E086F00A4F8C5F0600278FFC3E8956450025B
:10087D00A864886322C3E5409440E5419401E56393
:10088D005003140193046002F563227883E6F5208A
:10089D00120F1475E89012054075E89030EDFDA823
:1008AD00BDA9BE120FBA756E85756F00C3740013A6
:1008BD00FD7485606613FC74852CFC74003DFDECA5
:1008CD00FAEDFBC3E89AE99B4014E56E2485F56EBD
:1008DD00E56F3400F56FEA2CFAEB3DFB80E5AE6E6B
:1008ED00AF6FC3E56F13F9E56E13F8C3E913F9E8BC
:1008FD0013F87A03C3E913F9E813F8DAF7AA201A03
:10090D007009756E00756F000209281AEA6008EE0D
:10091D0028FEEF39FFDAF88E6E8F6F2275E8902280
:10092D007883E6FF30EDF9A8BDA9BE0570C3E5706B
:10093D0094084052757000E9FA79A0E76044EA70B6
:10094D0007E571601B020961C3E895716010E571DF
:10095D005006600C1402096D0460F902096DE57111
:10096D00F571C3946D401B7561C0C394044013753C
:10097D006180C39404400B756140C39404400375BA
:10098D00610075BB0E22EFC39401601F7485601B5F
:10099D00C3E894FFE994035012C3E8956EE9956F8F
:1009AD005009E561600C15610209BFE561F4600253
:1009BD000561A861C3E524985002A824C3E8956297
:1009CD00400AA862E562F460038562618825882685
:1009DD00E570B4070375BB1022743279A787F0A4B4
:1009ED00C5F0A2F733F8C3E895614002A8618822EB
:1009FD008824882588268864227540007541F02258
:100A0D00C2AF75C820A8CCA9CDAA3A30CF010A75BE
:100A1D00C824D2AFAB3BAC3C883B893CC3E89BF8C8
:100A2D00E99C206908F9306602611C4176AD3D8A6A
:100A3D003DF9EA9DFA600478FF79FFAE3EAF3F8B3A
:100A4D003E8C3FA83BA93CC3E89EF8E99FF9C3E55E
:100A5D004113FBE54013FAE82AF540E93BF5415017
:100A6D00067540FF7541FF41C3AA40AB41AC40AD97
:100A7D00417E047F02C3EB9404400D1E1FC3EB9413
:100A8D00084005206A021E1FC3ED13FDEC13FCDEAA
:100A9D00F7C3EA9CFAEB9DFBEF6009C3E913F9E894
:100AAD0013F8DFF7EA28FAEB39FB8A408B41500641
:100ABD007BFF8B408B41C3EB94025002D2663069B1
:100ACD00047F0341EE7892E6FFC3E537948240112F
:100ADD000FC3E53794A040010FC3EF940640027F8A
:100AED00057E02E541C4540FF9E541C454F0F8E523
:100AFD0040C4540F28F8C3E89EFAE99400FB40095E
:100B0D00C3EA9402EB940050047A02E4FB6168AAF4
:100B1D0040AB41EBC4FEEAC4540F4EFCC3EA9CFA51
:100B2D00EB9400FBC3E813C313F8EA28FAEB340087
:100B3D00FB8A408B41C3EB94024002C2667802EB04
:100B4D00C4FE7B00EAC4540F4EFAC3EA98FA40057E
:100B5D00C3940250027A027892E6FF306002616817
:100B6D00855192855293D26043E680C3E49AF8E4AE
:100B7D009BF930660261F4E8FAE9FBD3E913FDE86D
:100B8D0013FC88518952C3EF94036038EF20E00DB8
:100B9D00E82CF8E93DF9ECFAEDFB020BBDE828F87D
:100BAD00E939F9C3E82402F8E93400F97AFE7BFF4C
:100BBD00C3EF9403400E8A538B54884D894E8C4F4E
:100BCD008D508128885389548A4D8B4E8C4F8D5072
:100BDD003069127553F07554FF754FF07550FF75F0
:100BED0051F07552FF8128E8FAD3E813FC8851C300
:100BFD00EF94036020EF20E007E82CF8ECFA811465
:100C0D00E8282402F87AFEC3EF940340088A53883B
:100C1D004D8C4F812888538A4D8C4FE568C33350D6
:100C2D0002646BF5683060028132753402D2604324
:100C3D00E680E52D54066034A840A941C3E913F9B7
:100C4D00E813F8C3E913F9E813F8306904E924400F
:100C5D00F9C2AF53E67F759100C3E498F594E4991A
:0F0C6D00F595759104D26043E680D2AF22D26430
:100C7C00754300752000306C03752040020C99D22E
:100C8C0064754300752040306C0375200078017941
:100C9C0001206620E52D54066002C2647914E541FA
:100CAC00C313700104F8C39414400278143069041F
:100CBC00781B791B206010E543600C306903D53438
:100CCC0004D26DA144913A0543E59BF45440B52000
:100CDC0002A12E30690908C3E89940011881C0208F
:100CEC00640A08C3E8994002819981C0C264C2AF0A
:100CFC0053E67F7591003066127594007595F87502
:100D0C009104D26043E680D2AF8199E5417EFFC366
:100D1C00334005C3334001FEC3E49E759400F59542
:100D2C00A10BC3E53394015002819930640281997F
:100D3C00D802A14281C0C26DC2AF53E67F7591004B
:100D4C00855394855495759104854D92854E93D217
:100D5C006043E680D2AFE52D54066008206A020598
:100D6C0033020D80306D0D206C0A2064071581153F
:100D7C008102161B2278003064027801E53775F089
:100D8C0007A4F9E5F028F5F0E9A2F013A2F113A2FB
:100D9C00F213F537C394785003753778C3E537955C
:100DAC00384008D265C294C292C290306002A1B79A
:100DBC00854F92855093D26043E68022207D16C2E7
:100DCC00AF754202C293D295306202D290D2AF7507
:100DDC009F70020FB7C2AF754202C293D2913062BC
:100DEC0002D294D2AF759F70020FB7307243207D40
:100DFC0020C2AF754203900134757B08C290C2913A
:100E0C00306204D292C115D293D2AF759F00020FFB
:100E1C00B7C2AF754203900134757B08C294C2957A
:100E2C00306204D292C135D293D2AF759F20020F9B
:100E3C00B7207D17C2AF75420390010FC29030628C
:100E4C0002D292D2AF759F00020FB7C2AF754203A8
:100E5C0090010FC294306202D292D2AF759F2002E1
:100E6C000FB7207D16C2AF754204C295D291306285
:100E7C0002D292D2AF759F20020FB7C2AF75420457
:100E8C00C291D295306202D292D2AF759F00020FFE
:100E9C00B7307243207D20C2AF7542059001237597
:100EAC007B20C292C293306204D294C1BBD295D241
:100EBC00AF759F70020FB7C2AF75420590014575B3
:100ECC007B02C292C293306204D290C1DBD291D227
:100EDC00AF759F70020FB7207D17C2AF754205909A
:100EEC000105C292306202D294D2AF759F70020F8C
:100EFC00B7C2AF754205900119C2923062EBD29025
:100F0C00D2AF759F70020FB7207D16C2AF75420627
:100F1C00C291D293306202D294D2AF759F00020F6D
:100F2C00B7C2AF754206C295D293306202D290D24C
:100F3C00AF759F20020FB7307243207D20C2AF7572
:100F4C004201900145757B02C294C295306204D275
:100F5C0090E161D291D2AF759F20020FB7C2AF75ED
:100F6C004201900123757B20C290C291306204D261
:100F7C0094E181D295D2AF759F00020FB7207D17F7
:100F8C00C2AF754201900119C294306202D290D264
:100F9C00AF759F20020FB7C2AF754201900105C219
:100FAC0090306202D294D2AF759F00C2652290013C
:100FBC0003757B00C294C292C290C295C293C29137
:100FCC00C2622278807607087607087601087604D4
:100FDC000876FF0876FF08760A087602087601087C
:100FEC007601788C76010876000876B40876FF08CE
:100FFC0076FF0876FF0876030876FF0876010876F8
:10100C00FF0876250876D00876780876C808760426
:10101C000876FF08760108760008767A08760A08C2
:10102C0076010876010876000876FF0876002278AB
:10103C0087E6FFC2727888C27DE630E102D27DC2BB
:10104C007E7889E630E102D27EC3EF9402600875A7
:10105C008E01D273021068758E00C273227880E6FE
:0F106C00149000809378A5F67881E614900080A8
:10107B009378A6F67886E61490008D9378A7F67889
:10108B009FE6F87005756B0001AFC3E89411400241
:10109B007811E82828F56B256B256B28F56C256BEB
:1010AB002828F56D7886E6F539C394025003753917
:1010BB0002789CE67538FFB402037538A0B40303BD
:1010CB0075388278A3E61490009A93F566120FBADE
:1010DB0022227896E6FA7897E6FB7888E6B4030541
:1010EB00C3EB940EFB307F047A007BFFC3EB9AFCBF
:1010FB00C3948250027C827572000572EC8572F08B
:10110B00A4C3E5F0947D40F222D27F11DD12054F8E
:10111B0012054F7A007B007C10120545E55C2AFA1C
:10112B0074003BFBDCF37C04C3EB13FBEA13FADC2C
:10113B00F7FEC27F11DD22757C00757D00E5EF2087
:10114B00E6037520000520903FFFE5201460069014
:10115B001DFF1460009304600375EF1653D9BF7520
:10116B0081C043FF8012054075EF0643B203E5B320
:10117B00240220E70DF521E5E320E0068521B343AA
:10118B00E301120FBA7580FF75A40075F1DC75D4FD
:10119B00EF7590C075A53F75F23F75D5C075A6016B
:1011AB0075E241120FBAE4F8F6D8FD756801120F1B
:1011BB00CF12167278988673753001C2AF1205592B
:1011CB0012056912054F12057012054F12057712A1
:1011DB00054F121799120559120559120554C2AF32
:1011EB00757C00757D0078FA79FA308407D9FBD8C5
:1011FB00F7021C00113B116911DC11DD7898867325
:10120B00120FBA75881075890275C824759104750B
:10121B00D84075A82275B80275E690759B80759DB0
:10122B000075D10E75BC5875BB0E75BA1175E8807B
:10123B00120540D2AF12089875360053DACF207ED4
:10124B000343DA20307E0343DA1043DA01C2D8C2FB
:10125B0071120559D2617B037A0CE55B70077A0C2E
:10126B00DB030211E912054F2070030211E9C27072
:10127B00E55CC3940240E1E52F541F855E5DF55E8E
:10128B00B55DD5DAD5C26153DACF207E0343DA20C0
:10129B00307E0343DA10C2D8C27178A2E67008D24E
:1012AB0074E52F54E0F52FC27575290012055430E3
:1012BB007409C3E529940A4002D2751205457802D8
:1012CB003074027800C3E55C9840F0C2AF12056938
:1012DB00120569120569D2AF120559754C0012053A
:1012EB0045788CE6C3940150030213D6E530C394C2
:1012FB000150030213D6757CA5757DF1207435C39F
:10130B00E55C94FF50030213D6C2AF12057ED2AF39
:10131B00120554C3E55C940150EFC2AF120569127C
:10132B00054A120569D2AF120554C3E55C94FF4020
:10133B00E902181E7F05D27F11DD120554C2AFC220
:10134B007F11DDAE5CC3E55C947FD2AF500261E6EA
:10135B00120540C2AF12057ED2AFDFDA3114C3EEF5
:10136B0094057897F61205591217A17F0AD27F11AF
:10137B00DD120554C2AFC27F11DDAE5CC3E55C94D8
:10138B007FD2AF50E6120540C2AF12056912054A73
:10139B00120569D2AFDFD63114EE24037896F6F836
:1013AB007997E7C394824003985006E82482789794
:1013BB00F61205591216B41217D012055411DDC3CB
:1013CB00E55C94FF5002610102181E757C00757D6F
:1013DB0000C3E55C954C4003855C4C1205547801C9
:1013EB007988E7B403027805C3E55C98400241E9CC
:1013FB00C2AF12057E12057E12057ED2AF120559C1
:10140B00753000E4F531F5320531E531F4703F0507
:10141B0032789AE67819146012783214600D787D60
:10142B0014600878FA146003753200C3E5329840F3
:10143B001D120FBA1205401532753100789986735B
:10144B00C2AF12057ED2AF7898867312055412057F
:10145B004AE52A700530740221E97801207402787C
:0E146B0006C3E55C9840A1120554E52A700303
:101479000211E9C2AF120FBAE4F522F523F524F5FA
:1014890025F526F567D2AF7885E6C333F565E4F52A
:1014990044F545F546F547F548F570F52CF52DF574
:1014A9003775700875BB1012054012092930EDFD1A
:1014B900A8BDA9BEE97001F8887112092D757008D7
:1014C90075BB10113BC2AF7561FF1209E685226138
:1014D900852262852263D2AF7522017524017525A3
:1014E90001752601856069756A017888E6B4030784
:1014F900C27D307602D27DD268D269753300120F6F
:1015090014120F43120A06120A0D120A06120A0DC4
:10151900120A06120C8B12065F120D81120DC812E7
:101529000A0D120C7A306E031206FF2066031208A8
:1015390052306603120882120D81120DF7120A0D3C
:10154900120C8B306E0312073B120D81120E6E12B4
:101559000A0D120C7A306E03120799120D81120EC0
:101569009D120A0D120C8B306E031207F6120D81B3
:10157900120F14120A0D120929120C7A120D811276
:101589000F4312092D120A0D30692C856461856497
:1015990062856069756A0179187A0CC3E5339940E7
:1015A90009C269D26A8A350215C0C3E55C94014053
:1015B9000302151C021623306A1D206C1AE5351426
:1015C9007006C26AD26BA11CF535C3E55C94014073
:1015D9000302151C021623753600C3E55F9401400A
:1015E90009856462856069756A0178FA79A4E7609A
:1015F900027803C3E55F985021307404E52A601A24
:1016090078F0306C058564617820C3E54198500213
:10161900A11C0536E55C6002C126753600C2AF1211
:101629000FBA7887E6FE7602113B7887EEF6E4F585
:1016390022F523F524F525F526F565752C00752D7C
:1016490000D2AF120554120FBA78A4E66006D294FC
:10165900D292D290307406E52A700221E9788DE69B
:10166900C39401400241C6810E901A0D78201216CA
:10167900F6E520B4A50CA31216F6E520B45A030228
:101689001694120FCF1216B40216B3901A0378806B
:101699007B0A1216F6A308DBF9901A0F788C7B19CE
:1016A9001216F6A308DBF9901A2822C2AF121739CD
:1016B900121716901A00740E1216FBA3740712164D
:1016C900FBA374151216FB901A0378807B0A121675
:1016D900FAA308DBF9901A0F788C7B191216FAA372
:1016E90008DBF912174C12172A901A2822E493F6EC
:1016F90022E6438F01538FFDFFC3E583941C40010C
:1017090022EF857CB7857DB7F0538FFE22438F0288
:10171900438F01857CB7857DB7901A0DF0538FFCF7
:1017290022901A0D74A5D1FB901A0E745AD1FB227E
:101739007A3079D07820901A40D1F6E520F709A3BC
:10174900DAF7227A3079D0901A40E7D1FB09A3DA87
:10175900F922AB74A875BB01027980BB02027981B9
:10176900BB03027982BB04027994BB05027983BB6E
:1017790006027986BB07027992BB08027987BB0901
:1017890002799CBB0A027988BB0B027989E8F722A6
:101799007C05120559DCFB22C2AF120569120570DE
:1017A90012057712057E12054A1205691205701293
:1017B900057712057E12054A120569120570120590
:1017C9007712057ED2AF22C2AF12057E12057712BB
:1017D900057012056912054A12057E120577120570
:1017E9007012056912054A12057E120577120570F5
:1017F900120569D2AF22AE74AF75C2AF1205691274
:10180900056912056912054ADEF212057E12054ABA
:10181900DFF8D2AF221217A112179912179975740E
:10182900017575017576001217FF7C05AD5C12050F
:1018390059C3ED955C70F5C3E55C9401400AC3E5B5
:101849005C94FF403702186212175B1216B4121724
:10185900A1C2AF75EF16121799DCD10576C3E576EB
:0E1869009403500280C11217990575E574149E
:1018770090009F93F808C3E57598500280A8121747
:10188700991217990574C3E574940C500280941249
:0D1897000FCF1216B4C2AF75EF16121799DD
:0319FD0002114292
:101A00000E071507070104FFFF0A020101A55A018D
:101A100000B4FFFFFF03FF01FF25D078C804FF01DA
:091A200000FF0A010100FF00FFB4
:101A40002348694D6F64656C436F6F6C323241237C
:101A500023424C48454C4923463333302320202031
:101A60002020202020202020202020202020202076
:101C0000C2AFC2D353D9BF7581C043B20343FF8073
:101C1000752438752503B1DC7529A5752AF175E29F
:101C20004043F11053A4EF75D4FFD2847DFA7803BA
:101C300079E67C10752200752300901DE97B0675FE
:101C400024987525013084028145208408D8FBD969
:101C5000F9DCF781B7308408D8FBD9F9DCF781B714
:101C6000B19CE493A3C39A6004DDC381B7DBDBB10D
:101C70008E6002812E7B08E493FAA3B16FDBF87AC1
:101C800030B16F752200752300B18EEAFCEBFDC305
:101C9000ED94FE400EB18E8A278B28ED30E0048A49
:101CA000828B83B18E7AC270D8C3ED94FE601950D6
:101CB000CEBD002BEC600F7520007521FF7529004B
:101CC000752A000200008100A827A9280809D80465
:101CD000D90281DCB192EA89AAF281CE0D81A3C337
:101CE000ED94035053EDA2E092007AC5C3E58294CF
:101CF00000E583941C508A200010438F02438F011B
:101D00008529B7852AB7F0300029A827A92808090E
:101D1000438F01538FFDD804D902A133C3E58394C7
:101D20001C4003A3A11689AAE28529B7852AB7F02A
:101D3000A3A116538FFC817F7AC1BD030CE493A34A
:101D4000FAB153DCF8B14B817F8181AA22AB23B178
:101D50006FEBFAEA6222752608C3E52313F523E543
:101D60002213F52250066323A0632201D526EAB18F
:101D7000DCB1DC75260AEAF4200102D284300102CB
:101D8000C284B1DCC3134002C201D526EB22B1925A
:101D9000EAFB208402A192308402A197752608AE46
:101DA00024AF25C3EF13FFEE13FEB1E0B1DCC3EAAD
:101DB000133084024480FA30E703632201C3E52331
:101DC00013F523E52213F52250066323A0632201B5
:101DD000D526D9E52265236523F52222AE24AF2539
:101DE0000E0FDEFEDFFCD20122424C48656C6934E6
:071DF000373163F3300601F7
:00000001FF
